:100000000C941E060C94BC270C94E9270C9446060D
:100010000C94E8120C9446060C9446060C94460682
:100020000C9446060C9446060C9446060C94460620
:100030000C9446060C9446060C9446060C94460610
:100040000C9416280C9446060C94E72B0C942A2C3E
:100050000C9446060C9446060C9446060C944606F0
:100060000C9446060C9446064718A91888188B1855
:100070008E189118941897189A18A918A318DB19B4
:10008000DD19DD19DB19DD19DD19DD19DD19DD19C2
:10009000DD19DD19DD19DD19DD19DD19DD19DD19B0
:1000A0006119DD19DD19DD19DD19DD19D218DD1928
:1000B000DD19DD19DD19DD19DD19DD19DD19DD1990
:1000C000DD19DD19DD19DD19DD19DD196D196D1960
:1000D0006D196D196D196D196D196D196D19DD1980
:1000E000DD19DD19DD19DD19DD19D2186C196C194E
:1000F0006C196C19DD197A19801986198C199219E5
:1001000098199E19A419AE19B819C219CC19131946
:10011000D518DD19DD19DD19DD196119DD19DD19B4
:10012000DD19DD19DD19DD19DD19DD196B196B1903
:100130006B196B19DD197A19801986198C199219A6
:1001400098199E19A419AE19B819C219CC19131906
:10015000D518DD19DD19DD19DD196119101A101A0C
:10016000101A101A101A101A101A101A101A101A3F
:10017000101A101A101A261B261B261B261B261BBC
:10018000261B551A5F1A691A731AD01ADA1AE91A55
:10019000FA1A821C971CA31CAC1CBB1CE01CE91C9B
:1001A000321DFB1C45204B20512058206620882002
:1001B000A620456E746572206D656E752E2E2E001C
:1001C000546F67676C6564206D6963726F50504D42
:1001D00000546F67676C656420696E76657274653C
:1001E000642050504D2100546F67676C6564205443
:1001F00058206D7574696E672100546F67676C6570
:10020000642074656C656D65747279210050726F3D
:10021000746F636F6C206572726F72207769746897
:100220002052580054696D656F7574207768656E4B
:1002300020636F6E6E656374696E6720746F205201
:100240005800507265737320616E79206B65792058
:10025000746F2063616E63656C00436F6E6E6563DF
:1002600074696E6720746F2052582C20706F776508
:100270007220757020746865205258202877697440
:10028000682062696E6420706C7567206966206EF4
:100290006F74207573696E6720616C776179732064
:1002A00062696E642900546F67676C656420276912
:1002B0006D6D656469617465206F75747075742700
:1002C00000546F67676C65642027736C61766520E6
:1002D0006D6F64652700546F67676C6564202761E4
:1002E0006C776179732062696E642700546F676769
:1002F0006C65642050504D206368616E6E656C20A3
:100300006C696D69740053657420525353492069B8
:100310006E6A656374696F6E206368616E6E656C8A
:100320002028303D3D64697361626C652900536526
:10033000742050504D206D696E696D756D20737914
:100340006E630053657420626561636F6E20696E31
:1003500074657276616C0053657420626561636FC9
:100360006E2064656C617900536574206265616319
:100370006F6E206672657175656E637920696E2097
:10038000487A3A20303D64697361626C652C205074
:10039000783D504D52206368616E6E656C20782CFC
:1003A0002046783D465253206368616E6E656C202E
:1003B00078005365742050574D2073746F7020641B
:1003C000656C61792028302064697361626C6564B2
:1003D0002C20312D323535203D3D20302E317320FB
:1003E0002D2035306D696E29005365742050504DB5
:1003F0002073746F702064656C61792028302064EC
:10040000697361626C65642C20312D323535203D75
:100410003D20302E3173202D2035306D696E29003E
:10042000536574206661696C736166652064656CF0
:1004300061792028302064697361626C65642C20C6
:10044000312D323535203D3D20302E3173202D2089
:1004500035306D696E29002A2A2A2A2A2A2A2A2A50
:100460002A2A2A2A2A2A2A2A2A2A2A2A2A2A2A2AEC
:100470002A2A2A2A0052582041636B6564202D20C5
:1004800072657665727420737563636573736675E0
:100490006C21002A2A2A2A2A2A2A2A2A2A2A2A2AAD
:1004A0002A2A2A2A2A2A2A2A2A2A2A2A2A2A2A2AAC
:1004B000002A2A2A2A2A2A2A2A2A2A2A2A2A2A2AC6
:1004C0002A2A2A2A2A2A2A2A2A2A2A2A2A2A00528E
:1004D000582041636B6564202D20757064617465DC
:1004E000207375636365737366756C21002A2A2A0D
:1004F0002A2A2A2A2A2A2A2A2A2A2A2A2A2A2A2A5C
:100500002A2A2A2A2A2A2A2A2A2A0056616C696457
:100510002063686F69636573206172653A205B319F
:100520005D2D5B31365D20286368616E6E656C20E1
:10053000312D31362900536574206F7574707574D0
:1005400020666F7220706F727420005B585D2061AE
:10055000626F7274206368616E67657320616E6498
:10056000206578697420525820636F6E6669670051
:100570005B535D20736176652073657474696E6783
:100580007320746F205258005B525D20726576654F
:1005900072742052582073657474696E6773207486
:1005A0006F2064656661756C747300557365206EA9
:1005B000756D62657273205B312D445D20746F2010
:1005C0006564697420706F727473205B452D515D92
:1005D00020666F722073657474696E677300202DD6
:1005E00020726563656976657220636F6E66696700
:1005F000757261746F722C20727820737720000AF4
:100600000A6F70656E4C52536E67200053657420FC
:1006100073657269616C2062617564726174653AB8
:10062000200056616C69642063686F696365733A82
:100630002031202D20342B34202F2032202D203823
:10064000202F2033202D20382B34202F2034202D14
:10065000203132202F2035202D2031322B34202FF5
:100660002036202D20313600536574204368616E9A
:100670006E656C20636F6E6669673A20005365741F
:100680002044617461726174652028302D32293AEA
:10069000200053657420486F70206368616E6E653A
:1006A0006C7320286D61782032342C207365706162
:1006B000726174656420627920636F6D6D61732966
:1006C0002076616C69642076616C75657320312DCC
:1006D0003235353A2000536574206368616E6E656B
:1006E0006C2073706163696E6720287831306B48C5
:1006F0007A293A200053657420524620706F77653E
:10070000722028302D37293A200053657420524634
:10071000206D6167696320286865782920652E67E8
:100720002E20307844454144463030443A2000532E
:1007300065742062617365206672657175656E63AC
:10074000792028696E20487A293A20005B5A5D207A
:10075000656E746572207265636569766572206383
:100760006F6E66696775726174696F6E2075746902
:100770006C79005B465D20646973706C61792061FF
:10078000637475616C206672657175656E63696509
:10079000732075736564005B525D2063616C6375E3
:1007A0006C6174652072616E646F6D206B65792079
:1007B000616E6420686F70206C697374005B495DC2
:1007C000207265696E697469616C697A6520736508
:1007D0007474696E677320746F20736B65746368DB
:1007E0002064656661756C7473005B585D2072658A
:1007F00076657274206368616E67657320616E64EC
:100800002065786974206D656E75005B535D20739B
:100810006176652073657474696E677320746F20E8
:10082000454550524F4D20616E64206578697420B3
:100830006D656E7500557365206E756D62657273BA
:10084000205B302D395D20746F20656469742070E1
:100850006172616D657465727300202D2053797328
:1008600074656D20636F6E66696775726174696F18
:100870006E000A0A6F70656E4C52536E672000510D
:1008800029204F7574707574206265666F726520DB
:100890006C696E6B20283D465329203A2000502970
:1008A00020536C617665206D6F64652028657870D3
:1008B0006572696D656E74616C293A20004F29205C
:1008C00054696D65642042494E44206174207374FC
:1008D000617274757020203A20004E292050504DCE
:1008E000206F7574707574206C696D69746564200F
:1008F000202020203A200044495341424C454400E6
:100900004D292050504D205253534920746F20637D
:1009100068616E6E656C202020203A20004C2920F2
:1009200050504D206D696E696D756D2073796E63E1
:10093000202875732920203A200044495341424C15
:100940004544004B29204661696C736166652062ED
:100950006561636F6E20696E74762E2028312D32AA
:10096000353573293A20004A29204661696C736144
:10097000666520626561636F6E2064656C617920D5
:1009800028302D323535203D3E20313073202D204A
:100990003135306D696E293A200049292046616958
:1009A0006C7361666520626561636F6E206672714B
:1009B0002E203A200048292050574D2073746F7024
:1009C0002064656C6179202020202020203A2000BE
:1009D00047292050504D2073746F702064656C61FE
:1009E00079202020202020203A200046292046611E
:1009F000696C736166652064656C617920202020D4
:100A00002020203A200050574D206368616E6E65AB
:100A10006C200066756E6374696F6E3A2000292041
:100A2000706F72742000506F776572546F776572C3
:100A300000445446205548462033322D62697420C4
:100A400031306368004F70656E4C52536E67525878
:100A5000206D696E6920342F36636800466C7974A6
:100A6000726F6E2F4F72616E6765525820554846FF
:100A70002038636800525820747970653A20004429
:100A8000697361626C656400487A00203D3D200016
:100A900043616C63756C61746564207061636B6540
:100AA0007420696E74657276616C3A200042292068
:100AB0004D6963726F202868616C66292050504D23
:100AC000202020203A00412920496E766572746505
:100AD000642050504D20696E20202020203A0030A4
:100AE00029204D7574652062757A7A657220286DAB
:100AF0006F73746C79293A003929205365726961E2
:100B00006C2062617564726174653A00736D617224
:100B100074506F7274004672536B79005472616E38
:100B200073706172656E740044697361626C6564B0
:100B30000038292054656C656D657472793A2020FF
:100B40002020202020003729204368616E6E656CCC
:100B500020636F6E6669673A202000362920446161
:100B60007461726174652028302D32293A2020206A
:100B700000352920486F70206368616E6E656C7364
:100B80003A2020202020003429204368616E6E65C1
:100B90006C2073706163696E673A202000332920EE
:100BA000524620706F7765722028302D37293A2001
:100BB0002020003229205246206D616769633A2067
:100BC0002020202020202020003129204261736530
:100BD000206672657175656E63793A202020000089
:100BE00000000700020100000304060000000000EE
:100BF00000000001020408102040800102040810D7
:100C00002001020408102004040404040404040263
:100C10000202020202030303030303000000002395
:100C2000002600290000000000250028002B0000FD
:100C3000000000240027002A0000182D11241FBEE8
:100C4000CFEFD8E0DEBFCDBF13E0A0E0B1E0EEE330
:100C5000F0E602C005900D92A83CB107D9F716E066
:100C6000A8ECB3E001C01D92AC38B107E1F71CE07D
:100C7000CCE3DCE004C02297FE010E94212ECA339F
:100C8000D107C9F70E94542D0C941D300C9400001C
:100C900080917105813019F482E080937105809113
:100CA0007105833019F484E0809371050895A89547
:100CB0000895DC01ED91FC910190F081E02D099502
:100CC00008952091720530917305382748E0C901D5
:100CD000880F991F37FF06C09C0151E2252750E17C
:100CE000352701C09C01415091F730937305209343
:100CF0007205089588E38093740580E092ECA1E08A
:100D0000B0E08093750590937605A0937705B09336
:100D1000780587E08093810580E091EAACEBB3E34E
:100D20008093790590937A05A0937B05B0937C0519
:100D300085E0809382058DEE9EEFADEABEED809357
:100D40007D0590937E05A0937F05B0938005E3E831
:100D5000F5E080E090E0863028F4DC01AF54BC4F31
:100D60002C9101C020E0219301968831910599F7DB
:100D700082E080939B058AE080939C05089580E043
:100D80009EECADEEB4E38093B9059093BA05A093C1
:100D9000BB05B093BC0580E090E0A0E0B0E5809397
:100DA000BD059093BE05A093BF05B093C005E1ECCF
:100DB000F5E080E081938F5F8031E1F70895A0E056
:100DC000B0E0E5EEF6E00C94EA2DD82F0E946C28F6
:100DD0006115710581059105C9F30E948D2E109250
:100DE0007D0510927E0510927F0510928005C4E06B
:100DF000812C912C54018A94C0907D05D0907E0561
:100E0000E0907F05F0908005FE2CED2CDC2CCC24AE
:100E10000E94882EA50194010E94C92D6C0D7D1D94
:100E20008E1D9F1D60937D0570937E0580937F05C9
:100E300090938005C15001F7DD2309F450C003E809
:100E400015E0E801A12CB12C62E3C62ED12CE12CD7
:100E5000F12C8881882309F442C0B39419F40E94CC
:100E60007A063DC00E94882EA70196010E94C92DD6
:100E7000E1E0E60FA3E8B5E08A2F801B8A1520F495
:100E80008D918E13F9CFE9CF2091820530E0A0E15A
:100E9000B7E20E94612D9B01AC01AE2FB0E00E9431
:100EA000702D4090790550907A0560907B05709088
:100EB0007C05640D751D861D971D4090B9055090E9
:100EC000BA056090BB057090BC05461657066806CB
:100ED000790618F2E993A39488E1A812BACFCDB7A6
:100EE000DEB7E0E10C94062E8436910520F4BC01B7
:100EF00080E090E017C09C018E3B910528F42A55B4
:100F00003109AAE0B0E00CC0823D910528F4245BD1
:100F10003109A4E6B0E004C02D5C3109A8E5B2E0D7
:100F20000E94612DA4E6B0E09B01AC010E94702DEF
:100F3000089590E08C599F4F0E947407089561E0D6
:100F400089E00E94192960E089E00E9452290895F1
:100F5000892B11F061E001C060E089E00E94522914
:100F6000089560E08EE00E94192961E08FE00E9400
:100F7000192961E082E00E94192960E083E00E9463
:100F8000192961E084E00E941929089542E050E0A7
:100F900068E476E081E00E949C270895E3E0F0E0B9
:100FA00089E080935700E491E67081E0E63009F033
:100FB00080E00895CF93DF93C82F0E94CE07882347
:100FC00081F0DFB781E080937005F8940E945706A6
:100FD00088E180936000C0936000C1110E945706B1
:100FE000DFBFDF91CF9108958F929F92AF92BF9212
:100FF000CF92DF92EF92FF92CF93FC01C0A5EC2F2E
:10100000E770F0E0E758FC4FA081B0E0C7FF03C0F5
:1010100024E130E002C02FE030E0FC0197A183E141
:10102000989FF0011124E25CFE4F80809180A280A5
:10103000B380A20FB31F20E43FE14DE750E00E94D0
:101040007B2DA50194010E94A72D8C2F887149F456
:1010500069017A01E0EDCE0EE7E0DE1EE11CF11C35
:101060001BC0C7FF05C060E47AE88CE29EE004C0C4
:1010700060E07EEE8AEB9BE069017A01F8EBCF0E2F
:10108000FBE0DF1EE11CF11CA50194010E94A72DCD
:10109000C20ED31EE41EF51EC701B60169517C4F76
:1010A0008F4F9F4F28EE33E040E050E00E94A72D85
:1010B000A8EEB3E00E94702DCF91FF90EF90DF90EB
:1010C000CF90BF90AF909F908F9008958F3F9105E4
:1010D00051F048F0811522E0920738F081159340D5
:1010E00030F482E0089580E0089581E0089583E07F
:1010F0000895A0E0B0E0EFE7F8E00C94F32DEB01E9
:101100008A01B82FB695A0E028813981F8012083A3
:101110002A813B8121832C813D8122832E813F8145
:101120002383688179814A815B812C813D81EE81B5
:10113000FF819F2F9295990F990F907C272F2370F5
:10114000922B252F2370220F220F922B232F2370F7
:101150002295207F922BF80194830B5F1F4F2896D6
:10116000AF5FBA1788F680FF24C0888199810E94FA
:101170006608D82E8A819B810E946608E82E8C81A1
:101180009D810E946608F82E8E819F810E946608CC
:10119000F0E4DF9EA001112490E1E99E900111246A
:1011A000242B282BE4E0FE9EB0011124262BF8010D
:1011B0002083CDB7DEB7E7E00C940F2E803223E01A
:1011C000920708F1883E23E0920740F48F51934044
:1011D000E4E096958795EA95E1F70895803D27E04C
:1011E000920718F48C5D93400895883928E092079F
:1011F00068F4885C974074E0969587957A95E1F756
:101200008D509C4F089580E090E008958FEF93E01B
:1012100008958C30910540F4A4E0880F991FAA9599
:10122000E1F7885D9C4F0895843F23E0920718F40E
:1012300084529C4F0895811524E0920740F486570C
:10124000934FF4E0880F991FFA95E1F7089580E92C
:1012500098E008959C013695279525753575821B74
:10126000930B9C0123733373969587959695879579
:1012700083739373820F931F9C0154E036952795D7
:101280005A95E1F7280F391F2F703F7041E051E068
:10129000249FC001259F900D349F900D1124892F0C
:1012A00008955A98882319F00000419A02C000005E
:1012B000419800005A9A000008955A9A000086B199
:1012C0005A98000081700895CF93DF93D82F5C9ACD
:1012D0005A985C98C8E08D2F80780E945109DD0FE4
:1012E000C150C9F75A98DF91CF9108958F770E9426
:1012F00064090895CF93DF93D82FC8E08D2F8078AD
:101300000E945109DD0FC150C9F75A98DF91CF9162
:101310000895CF93DF935A98C8E080E0D82FDD0F6F
:101320000E945D098D0FC150C9F7DF91CF910895DB
:101330000E9476090E9489095C9A0895A1E0B0E0B4
:10134000E4EAF9E00C94F82D806869830E9464094E
:101350006981862F0E947A095C9A2196E2E00C94BA
:10136000142ECF93C0917D05C827E82FF0E0EC58EC
:10137000FA4F678589E70E949E096C2F8DE30E94D2
:101380009E096C2F82E40E949E09CF91089586E207
:101390000E9498090895CF93DF93EC016C818CE152
:1013A0000E949E096D818DE10E949E096E818EE1F1
:1013B0000E949E096F8180E20E949E09688581E2F9
:1013C0000E949E09698582E20E949E096A8583E2E5
:1013D0000E949E096B8584E20E949E096C8585E2CD
:1013E0000E949E096D858AE20E949E096E858EE6A6
:1013F0000E949E096F858FE60E949E09688980E79A
:101400000E949E09698981E70E949E096A8982E794
:101410000E949E09DF91CF910895CF92DF92EF92C3
:10142000FF92CF93DF936B017C01C11488E3D80650
:101430008CE9E8068CE1F80628F5C701B60120E83A
:1014400036E948E950E00E94A72DE901689760E875
:1014500079E687E69FEF0E94832D6C0D7D1D8E1D22
:101460009F1DF2E0660F771F881F991FFA95D1F72D
:1014700021E732E040E050E00E94A72DF22EE32E5B
:1014800080E421C0C701B60120E03DE241E351E024
:101490000E94A72DE901689760E073ED8EEC9EEF46
:1014A0000E94832D6C0D7D1D8E1D9F1D660F771F65
:1014B000881F991F21E732E040E050E00E94A72DED
:1014C000F22EE32E80E66C2F6F71680F85E70E9485
:1014D0009E096E2D86E70E949E096F2D87E70E9468
:1014E0009E09DF91CF91FF90EF90DF90CF9008950C
:1014F000682F8DE60E949E0908958F929F92AF9269
:10150000BF92CF92DF92EF92FF92CF93DF93D82FCB
:1015100083E00E94980980936F0584E00E949809F7
:1015200080936E0560E086E00E949E0961E087E09E
:101530000E949E096FE789E00E949E0965E08AE0AB
:101540000E949E0962E18BE00E949E0965E18CE0A9
:101550000E949E096DEF8DE00E949E0960E08EE082
:101560000E949E09DD2319F08BE291E008C02091D2
:101570009B0533E1239FC0011124825C9E4F0E9492
:10158000CB096CE880E30E949E096FE082E30E9431
:101590009E0962E483E30E949E0980919C0587FF77
:1015A00002C064E101C06AE084E30E949E096AE22D
:1015B00085E30E949E096DE286E30E949E0964ED28
:1015C00087E30E949E0960E088E30E949E0960E034
:1015D00089E30E949E09D11109C0C0907D05D09079
:1015E0007E05E0907F05F090800507C0C5E9CC2E10
:1015F000C1ECDC2EED2CCEEDFC2ECAE38F2C992411
:10160000AA24BB24682D8C2F0E949E09682D85E09A
:101610008C0F0E949E09FE2CED2CDC2CCC24CF5F7D
:10162000CE3361F76FEF83E40E949E096FEF84E48D
:101630000E949E096FEF85E40E949E096FEF86E489
:101640000E949E09DD2311F066E002C060918105D1
:101650008DE60E949E0960E089E70E949E096091E4
:1016600082058AE70E949E0960E083E70E949E0946
:1016700060E084E70E949E09D11109C0609179055C
:1016800070917A0580917B0590917C0504C060E0A3
:1016900071EA8CEB93E30E940D0ADF91CF91FF90EA
:1016A000EF90DF90CF90BF90AF909F908F90089574
:1016B00061E087E00E949E0964E28EE70E949E0935
:1016C00063E088E00E949E0960E088E00E949E0935
:1016D00065E087E00E949E0962E085E00E949E0925
:1016E00083E00E94980980936F0584E00E94980926
:1016F00080936E05089583E00E94980980936F059A
:1017000084E00E94980980936E0561E087E00E9462
:101710009E096AE070E080E090E00E948F280E94BD
:10172000580B00000895CF92DF92FF920F931F9302
:10173000CF93DF931F92CDB7DEB7082F162F8EE31E
:1017400099830E949E09F02EC02E9981D92E8C2D4E
:101750008F19811738F4F60161916F018FE70E94AC
:101760009E09F5CF64E085E00E949E0983E00E9417
:10177000980980936F0584E00E94980980936E0514
:101780000E946C2860936A0570936B0580936C05CA
:1017900090936D0569E087E00E949E0981E0809347
:1017A00071050F90DF91CF911F910F91FF90DF9006
:1017B000CF9008950F931F930E94930B8091710512
:1017C000813099F40E946C2800916A0510916B0594
:1017D00020916C0530916D05601B710B820B930B92
:1017E000603A76488140910548F3809171058130D7
:1017F00031F46DE971E080EE95E00E943B2A1F9183
:101800000F9108950F931F9380917105823021F4F9
:101810001092710581E020C0809171058130D9F46A
:101820000E946C2800916A0510916B0520916C054F
:1018300030916D05601B710B820B930B613A7648FA
:101840008140910540F061E087E00E949E0910927E
:10185000710582E001C080E01F910F910895CF9340
:10186000DF93EC014AE050E06D2F70E080EE95E0F0
:101870000E94092B6EE280EE95E00E940D2ABE01C7
:1018800084E0769567958A95E1F76F7077274AE04F
:1018900050E080EE95E00E94092B6EE280EE95E02C
:1018A0000E940D2ABE016F7077274AE050E080EE5B
:1018B00095E00E94092BDF91CF910895D82FC0E0C9
:1018C000CD1780F42C9A64E670E080E090E00E94EE
:1018D0008F282C9864E670E080E090E00E948F28CA
:1018E000CF5FEECF6CE271E080E090E00E948F2845
:1018F000E6CF0F931F93CF93DF93EC01062F15E0F4
:10190000115051F0CE010E940430081741F0602FB1
:10191000CE010E940C30F4CF82E00E945E0CDF9179
:10192000CF911F910F910895A0E0B0E0EAE9FCE0AB
:101930000C94EA2D482E562EC0E0D0E0612C712C7C
:10194000E12CF12C00E010E041100CC06090D205B9
:1019500086E4689E3001112459E1E52EF12C08EB54
:1019600015E01EC091E049120FC06090D205E6E478
:101970006E9E30011124FBE16F0E711C49E2E42ED2
:10198000F12C04E715E00CC082E0481209C028E100
:10199000622E77247394EE24E394F12C01ED15E08C
:1019A00043018C0E9D1E1092730510927205340136
:1019B000A62CA818B12CC30101966C01AE14BF046B
:1019C000A8F4A00EB11E511006C0C3010E9404303D
:1019D000F501808305C0F5016081C3010E94790C87
:1019E000F50180810E9461063601E2CFC3015110EA
:1019F00018C0C3010E940430B82EC6010E940430F2
:101A00002B2D30E0322F2227282B809172059091C8
:101A100073058217930779F4C0E0D0E055245394FE
:101A200093CF3601609173050E94790C6091720525
:101A3000C6010E94790CC05EDE4FC13E92E0D9071C
:101A400008F482CF852DCDB7DEB7E0E10C94062EE9
:101A500061E082E00E94940C089560E082E00E94C0
:101A6000940C8091D105853020F01092D1050E9410
:101A7000280D8091D1058093D205089561E080E022
:101A80000E94940C61E081E00E94940C089560E053
:101A900080E00E94940C882351F060E081E00E9475
:101AA000940C882321F080917405883349F00E94BA
:101AB000BF060E947A0681E00E94DF060E943E0D6A
:101AC0000895882319F069EA71E002C06DEA71E0B7
:101AD00080EE95E00E943B2A0895FF920F931F939A
:101AE000CF93DF9369EC7BE080EE95E00E94E729DD
:101AF0004091790550917A0560917B0570917C0544
:101B00002AE030E080EE95E00E94102B63EB7BE052
:101B100080EE95E00E94E72940917D0550917E0579
:101B200060917F057091800520E130E080EE95E0C6
:101B30000E94102B6DE97BE080EE95E00E94E72982
:101B40004AE050E06091810580EE95E00E94382BDC
:101B500067E87BE080EE95E00E94E7294AE050E0EC
:101B60006091820580EE95E00E94382B61E77BE072
:101B700080EE95E00E94E729C3E8D5E0F12C8E01C4
:101B800088818823A9F0FF2031F060EB71E080EEBE
:101B900095E00E940A2A21964AE050E0F80160810F
:101BA00080EE95E00E94012BF394F8E1FF12E7CF5D
:101BB00080EE95E00E94152A6BE57BE080EE95E0D3
:101BC0000E94E7294AE050E060919B0580EE95E095
:101BD0000E94382B66E47BE080EE95E00E94E729C6
:101BE000E0919C05E770F0E0EE0FFF1FEF57FC4F10
:101BF0006081718180EE95E00E943B2A61E37BE089
:101C000080EE95E00E94E72980919C0588718830DC
:101C100069F028F4811113C068E27BE00CC08031C8
:101C200041F0883161F46CE07BE005C06CE17BE061
:101C300002C066E17BE080EE95E00E94292A68EF11
:101C40007AE080EE95E00E94E72940917505509179
:101C5000760560917705709178052AE030E080EE96
:101C600095E00E94102B6FED7AE080EE95E00E94E7
:101C7000E7298091BD0580710E94610D66EC7AE0D4
:101C800080EE95E00E94E7298091BD0580740E9456
:101C9000610D6DEA7AE080EE95E00E94E72980917F
:101CA000BD0580720E94610D60E97AE080EE95E0EA
:101CB0000E94E72984E795E00E94F407AB01BC018C
:101CC0002AE030E080EE95E00E94F22A6BE87AE0AC
:101CD00080EE95E00E94E72984E795E00E94F407F2
:101CE0009B01AC0160E472E48FE090E00E94A72DBC
:101CF000BA01A9012AE030E080EE95E00E94F22AC4
:101D000068E87AE080EE95E00E94292ACDB7DEB738
:101D1000E5E00C94112E8F929F92AF92BF92CF92DA
:101D2000DF92EF92FF92811107C06FE77AE080EEB9
:101D300095E00E94292A2FC090E00E94740724E6B3
:101D400030E040E050E00E94A72DCA01B9012AE02E
:101D500030E040E050E00E94A72D49015A016B019C
:101D60007C012AE030E0B501A40180EE95E00E94FC
:101D7000F22A6EE280EE95E00E940D2A2AE030E021
:101D8000B701A60180EE95E00E94F22A63E780EE9B
:101D900095E00E944D2AFF90EF90DF90CF90BF908A
:101DA000AF909F908F9008951F93CF93DF9365E737
:101DB0007AE080EE95E00E94E72980919D058130D0
:101DC00041F46CE57AE080EE95E00E94292A10E06B
:101DD00050C0823019F465E47AE0F5CF843019F40C
:101DE00061E37AE0F0CF853091F766E27AE0EBCFFD
:101DF000C12FD0E0C930D1050CF441C068E3610FB8
:101E000080EE95E00E940D2A6EE17AE080EE95E08A
:101E10000E94E729BE016F5F7F4F4AE050E080EEED
:101E200095E00E94D12A63E17AE080EE95E00E947D
:101E3000E729C356DA4FE981E03218F566E07AE027
:101E400080EE95E00E94E7298981803130F06CE6D0
:101E500073E080EE95E00E940A2A69816F7070E05D
:101E60006F5F7F4F4AE050E080EE95E00E94DA2AF3
:101E70001F5F80914605181708F4BACF0FC061E3C1
:101E8000BECFEF70F0E0EE0FFF1FEF56FC4F60810A
:101E9000718180EE95E00E943B2AEACF6BEE79E0FB
:101EA00080EE95E00E94E7298091B5050E948B0E97
:101EB00060ED79E080EE95E00E94E7298091B6051B
:101EC0000E948B0E65EB79E080EE95E00E94E72999
:101ED0008091B7050E948B0E6AE979E080EE95E06B
:101EE0000E94E7294091AD055091AE056091AF0584
:101EF0007091B005411551056105710539F12AE070
:101F000030E080EE95E00E94102B67E679E080EEED
:101F100095E00E94E7298091B1050E949907AB01E5
:101F2000BC012AE030E080EE95E00E94102B63E4D3
:101F300079E080EE95E00E94E7294AE050E0609168
:101F4000B20580EE95E00E94382B06C06AE379E086
:101F500080EE95E00E94292A6DE179E080EE95E01F
:101F60000E94E7296091B3057091B4054AE050E002
:101F700080EE95E00E94222B60E079E080EE95E013
:101F80000E94E7296091AC05603450F470E06F5F07
:101F90007F4F4AE050E080EE95E00E94DA2A06C0CA
:101FA00067EF78E080EE95E00E94292A6AED78E0FC
:101FB00080EE95E00E94E7298091AB0580FF03C089
:101FC00062EB71E002C066EB71E080EE95E00E948A
:101FD0003B2A6DEB78E080EE95E00E94E729809146
:101FE000AB0582700E94610D6EE978E080EE95E0AD
:101FF0000E94E7298091AB0584700E94610D6FE714
:1020000078E080EE95E00E94E7298091AB0588702A
:102010000E94610DDF91CF911F9108950F931F933F
:10202000CF93DF93209143052F3FA9F56FEF75E024
:1020300080EE95E00E94E72981E893E00E942F0C52
:102040006EED75E080EE95E00E94E72980914405F1
:10205000909145050E942F0C6BEA75E080EE95E0AB
:102060000E94292A68E875E080EE95E00E94292AFE
:1020700060E775E080EE95E00E94292A6BE475E048
:1020800080EE95E00E94292A80EE95E00E94152AB4
:102090000E94D40E68C012160CF065C0332727FDCD
:1020A00030958091460590E0821793070CF45BC051
:1020B00066E375E080EE95E00E94E72960914305B4
:1020C000772767FD70954AE050E080EE95E00E942A
:1020D000DA2A6BE075E080EE95E00E94E72910E0D7
:1020E00008E2809147051817D0F5C12FD0E0CC0F3A
:1020F000DD1FC85BDA4F288130E0809143059927C6
:1021000087FD909501972817390739F56AEB71E03B
:1021100080EE95E00E940A2A4AE050E0602F80EEAF
:1021200095E00E94012B6EEB71E080EE95E00E943D
:102130000A2AE981EF70F0E0EE0FFF1FEF56FC4F27
:102140006081718180EE95E00E940A2A62EC71E064
:1021500080EE95E00E940A2A0F5F1F5FC2CF80EEDB
:1021600095E00E94152ADF91CF911F910F9108955C
:10217000FF920F931F93CF93DF93C3E8D5E0F12C29
:102180008E0188818823D1F164EC71E080EE95E0C6
:102190000E940A2A4AE050E06F2D80EE95E00E94EE
:1021A000012B61ED71E080EE95E00E940A2A2196F4
:1021B000F801208130E0A0E1B7E20E94612D9B018F
:1021C000AC01A0918205B0E00E94702DAB01BC0172
:1021D0008091790590917A05A0917B05B0917C055D
:1021E000480F591F6A1F7B1F2AE030E080EE95E000
:1021F0000E94102BF394F8E1FF12C2CFCDB7DEB7E7
:10220000E5E00C94112E1092DD0485E6EEEDF4E08D
:10221000DF011D928A95E9F70895CF93C82F8F3774
:1022200019F0883009F045C0E091DD04EE23D9F1C2
:10223000E150E093DD04F0E0E252FB4F10826DE0EC
:1022400070E080EE95E00E945906C0E08091DD04C8
:10225000C81760F4EC2FF0E0E252FB4F608170E0B1
:1022600080EE95E00E945906CF5FF0CF60E270E00B
:1022700080EE95E00E9459066DE070E080EE95E0FA
:102280000E945906C0E08091DD04C81778F5EC2F54
:10229000F0E0E252FB4F608170E080EE95E00E943A
:1022A0005906CF5FF0CF67E080EE95E00E940D2ADF
:1022B0001DC08B3119F40E9403111AC08D30C1F07A
:1022C0008A30B1F08091DD04843668F76C2F70E0BD
:1022D00080EE95E00E945906E091DD0481E08E0FCA
:1022E0008093DD04F0E0E252FB4FC08380E001C048
:1022F00081E0CF910895CF93C82F0E946C286093FE
:10230000C6047093C7048093C8049093C904C09313
:10231000DB04CC2329F040E051EE60E070E004C023
:1023200040E855E260E070E080EE95E00E94972C76
:10233000CF9108959091CA04492F4F7050E0BA018F
:102340006F5F7F4F292F30E0E4E035952795EA95C0
:10235000E1F76217730759F0FA01E553FB4F8083E9
:1023600081E0890F8F70907F892B8093CA04089534
:102370006EE770E080EE95E00E9459060895A3E1B3
:10238000B1E0E5ECF1E10C94EB2DE3E8F5E0712C24
:102390008191882321F0739428E17212F9CF65EDC1
:1023A00071E080EE95E00E943B2A4AE050E0672D04
:1023B00080EE95E00E94382B80E00E947D0A0E940A
:1023C000580B8E010E5F1F4FC12CD12C7601C39488
:1023D00066246A945C2C0E9460284B015C01209169
:1023E000820530E0A0E1B7E20E94612D9B01AC01C3
:1023F000C701B6010E94832D2091790530917A059D
:1024000040917B0550917C05620F731F841F951FBF
:102410002091B9053091BA054091BB055091BC059A
:10242000261737074807590718F4F801608225C0B6
:102430008C2D0E94B10961E070E080E090E00E9484
:102440008F28F80110820E946028681979098A098A
:102450009B09643F71408105910540F40E94C709C2
:10246000F8019081981778F78083EDCF50FE03C074
:102470002B982C9A02C02B9A2C982FEFC21AD20AB2
:10248000E20AF20A0F5F1F4F8FEFC816D104E10472
:10249000F10409F09FCFCE019395FC01D82E7FEF78
:1024A00068EC2E2F281B271510F051E056C0DE01D6
:1024B000129651E02FEF41E03D91321710F0322F8C
:1024C00001C0452F5F5F5F3F11F0232FF5CF419390
:1024D000242F30E0A1E0B0E0AC0FBD1FA20FB31F6E
:1024E0005C93413079F0DE01A20FB31F5C93423060
:1024F00049F0AFEFBFEFAC0FBD1FA20FB31F6C933E
:102500004E3F78F6A2E0B0E0AC0FBD1FA20FB31FA4
:102510007C934D3F30F6A3E0B0E0AC0FBD1FA20F9F
:10252000B31F6C93BECF452F242F30E0FC01E20F88
:10253000F31F6081AFEFB0E0AC0FBD1FA20FB31F60
:102540002C91621748F44150DC01A40FB11D2C916D
:1025500020836C934111E8CF5F5F571520F3372D2F
:10256000369520E0231770F4DC01A20FB11D4C91C9
:10257000522F530FFC01E50FF11D50815C934083F6
:102580002E5FF0CFF3E8EF2EF5E0FF2E8C01802FC9
:102590008D19871598F4F801C1908F014AE050E039
:1025A0006C2D80EE95E00E94012B6CE280EE95E0B0
:1025B0000E940D2AF701C1927F01E9CF80EE95E0DC
:1025C0000E94152A81E0CD5EDE4FEFE00C94072ECD
:1025D0001F920F920FB60F9211240F931F932F93F8
:1025E0003F934F935F936F937F938F939F93AF939B
:1025F000BF93EF93FF934091BD055091BE0560914D
:10260000BF057091C00586B18A019B010074112736
:102610002227332785FB882780F990E0A0E0B0E0EF
:10262000081719072A073B0709F468C0809184003E
:102630009091850010928500109284002091A7044B
:1026400021115CC045FD02C096958795853C29E027
:102650009207C0F180910A0190E0A0E0B0E00CE1A7
:1026600076956795579547950A95D1F74115510588
:102670006105710521F441E050E060E070E0481729
:1026800059076A077B07D8F480910A018F3FB9F098
:1026900040E080910A01481780F4842F90E0880F71
:1026A000991FFC01E957FB4F20813181FC01E55F57
:1026B000FE4F318320834F5FECCF1092A80410921D
:1026C0000A011CC08D3B22E09207A8F020910A016C
:1026D000203188F410910A0121E0210F20930A0192
:1026E0000E94DE08E12FF0E0EE0FFF1FE957FB4FDD
:1026F0009183808303C08FEF80930A01FF91EF9154
:10270000BF91AF919F918F917F916F915F914F9109
:102710003F912F911F910F910F900FBE0F901F901F
:10272000189583E0809380008AE1809381008FEF89
:102730009FEF909389008093880010926F0080E251
:1027400080936C00E8E6F0E08081826080830895E9
:102750000E942D0D8091D205843011F41092D20583
:1027600008956F3018F086958058089589E0689F25
:10277000802D11240895A0E0B0E0E1ECF3E10C9489
:10278000F22DC82F0E946C28009138041091390452
:1027900020913A0430913B046B017C01C01AD10AAC
:1027A000E20AF30A9701860149E8C41643E1D40618
:1027B000E104F10410F010923C046093380470932B
:1027C000390480933A0490933B042091A7048FEF3F
:1027D000820F8230D8F5E0913C04EE2309F44EC11B
:1027E000E13011F482E0B8C1E03108F034C181E099
:1027F0008E0F80933C04F0E0E957FB4FC08380319B
:1028000009F0ACC1E9E8F4E0213029F4A181A695F2
:10281000A695808108C080819181A92FA695A69553
:10282000A69596958795A03148F4B0E090E0AA0F60
:10283000BB1FA55FBE4F11969C938E931092A80468
:10284000329684E0E739F807F9F688C1233009F0B9
:1028500005C1E0913C04E11104C0CF3009F07EC114
:102860000DC1E83148F481E08E0F80933C04F0E024
:10287000EA57FB4FC08372C1E83109F0ECC0C111C7
:10288000EAC040E050E0ABE0CA01B3E0880F991F16
:10289000BA95E1F7A49F9001A59F300D1124F9018D
:1028A000E957FB4F6081E1817E2F777075956795C1
:1028B000FC01EE0FFF1FE55FFE4F71836083F9019E
:1028C000E857FB4FB081B695B695B695E181FE2FDE
:1028D000F295FF0FF07E6F2F6B2BE695E695E69550
:1028E0007E2F777075956795FC01EE0FFF1FE35FF4
:1028F000FE4F71836083F901E757FB4FB081B295BA
:10290000B695B695B370C181DC2FDD0FDD0F6D2F4D
:102910006B2BC295C695C695C370E281E170EE0F30
:10292000EE0F7E2F7C2B75956795FC01EE0FFF1F38
:10293000E15FFE4F71836083F901E557FB4FB08182
:10294000B695E181FE2FF795FF27F7956F2F6B2B3B
:10295000E6957E2F777075956795FC01EE0FFF1F4A
:10296000EF5EFE4F71836083F901E457FB4FB08146
:10297000B295BF70E181FE2FF295F07F6F2F6B2B28
:10298000E295EF707E2F777075956795FC01EE0FDD
:10299000FF1FED5EFE4F71836083F901E357FB4F2C
:1029A000B081BB1FBB27BB1FC181DC2FDD0F6D2F8B
:1029B0006B2BCC1FCC27CC1FE281E370EE0F7E2F58
:1029C0007C2B75956795FC01EE0FFF1FEB5EFE4FAC
:1029D00071836083F901E157FB4FB081B695B695DD
:1029E000E181FE2FF295FF0FFF0FF07C6F2F6B2B15
:1029F000E695E6957E2F777075956795FC01EE0F4D
:102A0000FF1FE95EFE4F71836083F901E057FB4FC2
:102A100020812295269527703181E32FEE0FEE0F4E
:102A2000EE0F6E2F622B732F7295769577707595DA
:102A30006795FC01EE0FFF1FE75EFE4F7183608319
:102A40004F5F5F4F4230510509F01ECF80919D04CA
:102A500083FF1092A80410923C0480C0243009F037
:102A60007DC060913C0461110BC0C83AB1F4109272
:102A700073051092720588EA0E94610681E06CC0BD
:102A8000613019F4C093370404C0623031F4C0934C
:102A900036048C2F0E9461065AC0E09136042E2F16
:102AA00030E0220F331F462F50E0C90102968417F1
:102AB00095073CF0633268F7FA01EC57FB4FC0838F
:102AC000E8CF2D5F3F4F8C2F90E0609172057091A1
:102AD00073054217530749F4982F882786279727AD
:102AE000909373058093720532C06817790769F572
:102AF00080913704813049F5E13118F080E180930D
:102B00003604F0903604C8E8D4E000E010E00F1579
:102B1000D0F4FE013197808190E0982F882728819A
:102B2000822B43E0969587954A95E1F70E94DE084F
:102B3000F801EE0FFF1FE55FFE4F918380830F5F6B
:102B40001F4F2296E4CF1092A80410923C0480916B
:102B50003C04882319F08F5F80933C04CDB7DEB727
:102B6000E8E00C940E2EE82FF0E0E854FA4FE185EF
:102B7000E03150F4F894F0E0EE0FFF1FE55FFE4FF8
:102B8000808191817894089580E092E00895A2E296
:102B9000B0E0EDECF5E10C94E82D9E012F5F3F4F86
:102BA00080E1D9011D928A95E9F763E072E080EE39
:102BB00095E029A33AA30E943B2A0E947B0B1D8A21
:102BC0001E8A1F8A188E312C212C00E0812C912C1A
:102BD0005401412C74E7572E7BE8672E72E3772E61
:102BE000E0E5CE2EE3ECDE2EE12CF12C84EF91E03B
:102BF000A0E0B0E08D8F9E8FAF8FB8A380E09EECF9
:102C0000ADEEB4E3898F9A8FAB8FBC8F80E094E7F1
:102C1000ABE8B2E3898B9A8BAB8BBC8B80EE95E0F3
:102C20000E944F2B892B09F4E1C080EE95E00E94B1
:102C30007C2B9C0133272C32310509F442C0ACF4C3
:102C40002332310509F0ABC019821A821B821C8223
:102C50001D821E821F82188619861A861B861C8674
:102C60001D861E861F86188A60C02434310529F00F
:102C70002335310509F4B2C092C064E480EE95E0DA
:102C80000E940D2A2AE030E040E054E76BE872E34E
:102C900080EE95E00E949B2A6CE280EE95E00E9417
:102CA0000D2A2AE030E040E05EEC6DEE74E380EE49
:102CB00095E00E949B2A6CE280EE95E00E944D2AEE
:102CC000ADCF0F5F043009F0A9CF29813A814B8144
:102CD0005C81A8EEB3E00E94702D698B7A8B8B8BA0
:102CE0009C8B2D813E814F8158850E94702D698F6C
:102CF0007A8F8B8F9C8F29853A854B855C852D8FAC
:102D00003E8F4F8F58A32D853E854F8558890E9451
:102D1000702D6B017C0160323EE4730781059105E3
:102D200030F462E38CE10E949E0900E077CF6033CB
:102D300045E774078105910510F462E2F3CF603432
:102D40005CE975078105910510F466E2EBCF80E53B
:102D5000C81683ECD806E104F10410F462E1E2CF76
:102D600090E6C9169AEED906E104F10410F465E183
:102D7000D9CFA0E7CA16A1E1DA06A1E0EA06F1047C
:102D800010F461E0CFCFB0EACB16B6E8DB06B1E0D5
:102D9000EB06F10410F463E0C5CF65E0C3CF10ED9E
:102DA000180F1A3008F03ACFE1E0F0E0EC0FFD1F09
:102DB00024E0029FE00DF11D112420813181428128
:102DC0005381AAE0B0E00E94702D610F711D811D3A
:102DD000911D608371838283938320CF49885A88B1
:102DE0006B887C88812C912C540118CF811491041C
:102DF000A104B10489F4C301B2010E940D0A61E08B
:102E000070E080E090E00E948F281D8A1E8A1F8A51
:102E1000188E312C22242A948D8D9E8DAF8DB8A1D1
:102E200088169906AA06BB06D0F40E94C7092D8908
:102E30003E894F89588D280F311D411D511D2D8B05
:102E40003E8B4F8B588F381608F4382E821508F4B5
:102E5000282E3FEF831A930AA30AB30A56C0C30170
:102E6000B20128EE33E040E050E00E94A72DBA0105
:102E7000A9012AE030E080EE95E00E94F22A6CE29F
:102E800080EE95E00E940D2A4AE050E0632D80EE2E
:102E900095E00E94012B6CE280EE95E00E940D2AE5
:102EA0006D897E898F89988DA50194010E94A72D37
:102EB000BA01A9012AE030E080EE95E00E94F22AF2
:102EC0006CE280EE95E00E940D2A4AE050E0622D0F
:102ED00080EE95E00E94012B6CE280EE95E00E946E
:102EE0004D2A4C0C5D1C6E1C7F1C898D9A8DAB8D00
:102EF000BC8D84159505A605B70520F449885A8828
:102F00006B887C88812C912C540129893A894B89C2
:102F10005C89283E33404105510509F07FCEA296D9
:102F2000E2E10C94042EACE1B0E0E9E9F7E10C94A5
:102F3000F22D0E946C286B017C0181E00E947D0AC9
:102F400014E703E0198361E0CE0101960E94DA0BD9
:102F5000009371050E94580B6AEF70E080E090E0EA
:102F60000E948F2880917105833089F480EE95E06E
:102F70000E944F2B892B59F40E946C286C197D09F3
:102F80008E099F096038734C894C9140D8F280912A
:102F90007105833009F44FC08FE70E9476090E94C3
:102FA00089098983843511F083E05CC00E94890916
:102FB00010924405809345050E948909209144059B
:102FC00030914505280F311D309345052093440568
:102FD0000E948909809346050E94890980934705CC
:102FE000813110F7F12C0F2D10E08091470590E012
:102FF000880F991F0817190740F40E948909F801E2
:10300000E85BFA4F8083F394EECF80E7898361E039
:10301000CE0101960E94DA0B83E0809371050E9435
:10302000580B62E370E080E090E00E948F2880916E
:103030007105833011F482E015C08FE70E94760994
:103040000E9489098983803509F0AECF0DE915E02A
:103050000E948909F80181938F01F5E0083B1F0761
:10306000B9F781E06C96E8E00C940E2E8091430550
:10307000992787FD9095A92FB92FFC013196EB3048
:10308000F10508F066C0EC5CFF4F0C941F2E62E760
:1030900078E080EE95E00E94292A81E893E00E9482
:1030A0002F0C6AE578E080EE95E00E94292A65E31E
:1030B00078E080EE95E00E94292A6BE078E080EECF
:1030C00095E00E94292A6AEE77E080EE95E00E9462
:1030D000292A6DEB77E080EE95E00E94292A67E9C6
:1030E00077E080EE95E00E94292A63E777E080EEA2
:1030F00095E00E94292A6CE477E080EE95E00E943A
:10310000292A80EE95E00E94152A0E946D0D21C0AB
:103110006FE277E01AC06AE077E017C065EF76E00B
:1031200014C066ED76E011C062E976E00EC06DE78E
:1031300076E00BC068E676E080EE95E00E94292AF2
:1031400062E276E002C06CE076E080EE95E00E94FC
:10315000292A6AE070E080E090E00E948F2880EEEB
:1031600095E00E944F2B892B29F080EE95E00E947C
:103170007C2BF5CF0895ACE1B0E0E1ECF8E10C94E4
:10318000F22D909143059F3F09F023C1482F50E055
:10319000FA013A97EF36F10508F00FC1E15CFF4FF5
:1031A0000C941F2E60E172E0A0C06CE172E080EE32
:1031B00095E00E943B2A85E789838BE1EDE9F5E004
:1031C000DE01129601900D928A95E1F76CE1CE0135
:1031D00001960E94DA0B0E94580B83E080937105E0
:1031E00068EC70E080E090E00E948F28809171058B
:1031F000843009F0E2C08FE70E9476090E948909B5
:103200008983853509F0D9C06DEE74E080EE95E0D4
:103210000E94292A6FEC74E080EE95E00E94292A32
:1032200061EB74E096C064E372E080EE95E00E948A
:103230003B2A89E6898361E0CE0101960E94DA0B80
:103240000E94580B83E08093710568EC70E080E089
:1032500090E00E948F2880917105843009F0ADC004
:103260008FE70E9476090E94890989838E010E5F8B
:103270001F4F7E014DE1E40EF11C0E948909F80107
:1032800081938F01EE15FF05C1F78BE1FE013296A8
:10329000ADE9B5E001900D928A95E1F78981893415
:1032A00009F08BC063E974E080EE95E00E94292A62
:1032B00065E774E080EE95E00E94292A67E574E0F6
:1032C00048C06EE472E080EE95E00E943B2A8EEFEB
:1032D0008093430572C08052875080539091460579
:1032E000981708F066C06DE572E080EE95E00E94E8
:1032F0003B2A63C084E18093430560E274E029C007
:1033000085E18093430569EE73E023C086E18093F5
:10331000430562EB73E01DC087E18093430568E6D7
:1033200073E017C088E18093430567E573E011C03F
:1033300089E18093430563E473E00BC08AE18093E5
:1033400043056EE273E005C08BE18093430566E0C0
:1033500073E080EE95E00E94292A2FC06CEE72E0A7
:1033600080EE95E00E94292A8091AB0591E01DC076
:1033700066ED72E080EE95E00E94292A8091AB050F
:1033800092E013C061EC72E080EE95E00E94292A81
:103390008091AB0594E009C066EA72E080EE95E0AA
:1033A0000E94292A8091AB0598E089278093AB057C
:1033B0008FEF809343050E940E1080EE95E00E94EF
:1033C0004F2B892B09F45AC180EE95E00E947C2B8B
:1033D000F4CF0E940D11882309F450C18091DD04BF
:1033E000811104C08FEF8093430540C140E050E05D
:1033F00060E070E08EED94E00E94962E40914305CF
:10340000042F112707FD1095212F312FF801319737
:10341000EB31F10508F01AC1E255FF4F0C941F2E55
:10342000552747FD50952091460530E02417350774
:103430000CF40CC18B019C010150110921093109C7
:10344000003211052105310558F0C0904705E9E427
:10345000F5E0F12CD12CA8E2EA2E415051090FC021
:10346000FA01E356FA4F61506083D8C0DF0111972B
:103470002C9130E02417350729F0F3943296FC1094
:10348000F5CFCAC00E2D10E020E030E00617170778
:103490002807390741F42081DA01A356BA4F119663
:1034A0002C93DD24D394E394E8CF6F3F710581051D
:1034B000910511F008F0CAC06093B505AFC06F3F29
:1034C00071058105910511F008F0C0C06093B60543
:1034D000A5C06F3F71058105910511F008F0B6C0D8
:1034E0006093B7059BC02091DE0420622037E9F489
:1034F00040E050E060E070E08FED94E00E94962E96
:103500009B01AC01DC01CB010197A109B10908972E
:10351000A105B10508F0ADC0A4EDB0E30E94702D87
:103520006A5E7C4A8A46954E24C02636E9F440E01D
:1035300050E060E070E08FED94E00E94962E9B01D9
:10354000AC01DC01CB010197A109B1090797A105E5
:10355000B10508F08EC0A8EAB1E60E94702D645E45
:103560007C438E46944E05C0611571058105910519
:1035700071F08B019C0114572B4832430130FAE55E
:103580001F07F2E62F07F2E03F0708F05FC06093E5
:10359000AD057093AE058093AF059093B0053EC026
:1035A0006F3F71058105910511F008F04FC06093E0
:1035B000B10534C08B019C01015011092109310969
:1035C0000F3F11052105310508F040C06093B20599
:1035D00025C08B019C01045C1940210931090D347F
:1035E0004DE114072105310528F47093B40560936B
:1035F000B30514C0611571058105910521F48FEFA4
:103600008093AC050BC06134710581059105F0F420
:1036100061506093AC0502C0DD20C1F08091DC04F4
:1036200081111AC080917D0590917E05A0917F0542
:10363000B09180050196A11DB11D80937D059093E9
:103640007E05A0937F05B093800506C06FE672E00B
:1036500080EE95E00E943B2A0E9403118FEF809339
:1036600043056AE080EE95E00E944D2A0E940E100C
:1036700005C061E070E080E090E07BCF6C96E8E010
:103680000C940E2E6AE572E080EE95E00E94292AE5
:1036900062E472E080EE95E00E94292A80EE95E0D7
:1036A0000E944F2B892B31F080EE95E00E947C2BFD
:1036B0000E94BB180E949317823029F0833051F486
:1036C0006DE072E002C064E272E080EE95E00E947C
:1036D000292A08958FEF809343051092DC040E94FD
:1036E0000E10809143058E3F69F080EE95E00E94B8
:1036F0004F2B892BB1F380EE95E00E947C2B0E942A
:10370000BB18EFCF08950F931F93109143051F3FF0
:1037100009F0D2C0893409F457C000F5883309F4A0
:1037200069C058F4803309F477C008F061C08B3168
:1037300009F440C08132B1F1B9C0813409F487C0C5
:1037400030F4893309F466C0803461F1AFC082344B
:1037500009F48EC0863409F448C0A8C0823609F442
:1037600087C078F4883531F128F48235C1F183358A
:10377000E1F09CC08A3509F494C0813609F467C031
:1037800095C0823761F128F4863679F18936E1F007
:103790008DC0883779F08A3709F483C0833709F000
:1037A00085C003C060E172E015C00E943E0D6DE867
:1037B00072E004C00E94470D67EA72E080EE95E077
:1037C0000E943B2A8EEF70C00E947A060E94BF06BC
:1037D00066EC72E080EE95E00E943B2A67C081E0D3
:1037E0000E94DF066FED72E0F5CF0E94B8105EC058
:1037F00080535AC06AEF71E080EE95E00E94292A5A
:1038000090919C0588E0890F8871977E892B809321
:103810009C051AC089E048C067EE71E080EE95E033
:103820000E94292A8091BD059091BE05A091BF05F7
:10383000B091C00520E182278093BD059093BE051D
:10384000A093BF05B093C005109343052FC061ED51
:1038500071E080EE95E00E94292A8091BD0590914B
:10386000BE05A091BF05B091C00540E4842710C0FB
:1038700060EC71E080EE95E00E94292A8091BD0500
:103880009091BE05A091BF05B091C00520E28227AE
:103890008093BD059093BE05A093BF05B093C0056E
:1038A00002C00E94421B8FEF809343058091430525
:1038B0008E3F09F0D4C0DDC00E940D11882309F4A9
:1038C000D8C08091DD04811104C08FEF809343053F
:1038D000C6C040E050E060E070E08EED94E00E94F1
:1038E000962E00914305112707FD1095212F312FAA
:1038F000F8013197E930F10508F0B4C0E753FF4F04
:103900000C941F2E8B019C01015014472B4832430D
:103910000F3F19452246324008F0A4C06093790554
:1039200070937A0580937B0590937C0577C06093B4
:103930007D0570937E0580937F059093800581E0DF
:103940008093DC046BC0683071058105910508F037
:1039500089C06093810562C08B019C0101501109EF
:10396000210931090A3011052105310508F07AC015
:103970006093820553C060EB71E08EED94E00E948D
:10398000D02F10E0009799F00E94AA2F009779F0AD
:10399000183130F4E12FF0E0EC58FA4F87871F5FC1
:1039A00060EB71E080E090E00E94D02FEBCF183107
:1039B000A8F5E12FF0E0EC58FA4F17861F5FF7CF1C
:1039C000653071058105910508F04CC060939B0539
:1039D00025C08B019C0101501109210931090630D4
:1039E000110521053105F0F520919C05287F262B36
:1039F00020939C0513C08B019C01015011092109E2
:103A000031090115124C2140310560F560937505AF
:103A10007093760580937705909378058091DC0408
:103A2000811113C080917D0590917E05A0917F0545
:103A3000B09180050196A11DB11D80937D059093E5
:103A40007E05A0937F05B09380050E9403118FEF40
:103A5000809343056AE080EE95E00E944D2A0E9423
:103A6000361807C06FE672E080EE95E00E943B2AB0
:103A7000ECCF1F910F9108958FEF80934305109223
:103A8000DC040E943618809143058E3F69F080EE79
:103A900095E00E944F2B892BB1F380EE95E00E94B8
:103AA0007C2B0E94831BEFCF6AE070E080E090E007
:103AB0000E948F2880EE95E00E944F2B892B29F0E1
:103AC00080EE95E00E947C2BF5CF0895CF93C82F10
:103AD000682F80EE95E00E94A92B909168059C27A5
:103AE00090936805CF910895A1E0B0E0EAE7FDE189
:103AF0000C94F82D99830E94661D9981892F0E944C
:103B0000661D2196E2E00C94142E1F93CF93DF9351
:103B1000182FEB011092680565EB70E080EE95E0E0
:103B20000E94590662E670E080EE95E00E94590618
:103B3000812F0E94661DCE010E94741DDF91CF91DE
:103B40001F9108956091680580EE95E00E94A92B71
:103B50000895A1E2B0E0EFEAFDE10C94F42D7B01C1
:103B60008A018C3009F453C108F040C0863009F452
:103B7000BCC018F5833009F491C070F4813009F4A9
:103B800072C0823009F048C26BE170E082E00E94AE
:103B9000851D0DE915E078C0843009F487C08530B3
:103BA00009F03AC26091470570E0660F771F85E023
:103BB0000E94851D08E415E086C0893009F4A7C07D
:103BC00070F4873009F49BC0883009F025C261E0A9
:103BD00070E088E00E94851D8091D20523C28A3062
:103BE00009F4CAC08B3009F4F2C016C28A3609F44F
:103BF00075C1D8F4873609F43AC138F4853609F42A
:103C00000EC1863609F41FC107C2883609F437C1D0
:103C1000893609F001C261E070E089E60E94851DE5
:103C20000E947A060E94BF06F5C18D3609F4D4C100
:103C300038F48B3609F491C18C3609F49AC1ECC181
:103C40008E3609F4DCC1873C09F0E6C161E070E022
:103C500087EC0E94851D81E00E94661D0E94A21DC6
:103C600010926905E3C169E270E081E00E94851D60
:103C700004E715E0F80181918F010E94661DF5E0CF
:103C80000D391F07B9F7D0C1F80181918F010E944A
:103C9000661DF5E0083B1F07B9F7C6C161E070E09B
:103CA00083E00E94851D0E949317BCC161E070E013
:103CB00084E00E94851D81E00E94661D0E94A21D75
:103CC0000E94C715B3C18091470590E0880F991FE6
:103CD0009801285435402817390708F0A5C1F80184
:103CE00081918F010E94661DEECF62E070E086E058
:103CF0000E94851D81E893E00E94741D95C161E0DA
:103D000070E087E00E94851D809146058BC186E6A4
:103D1000898361E0CE0101960E94DA0B0E94580B64
:103D200083E08093710568EC70E080E090E00E9491
:103D30008F28809171058430D9F48FE70E9476092D
:103D40000E9489098983863469F460E270E089E021
:103D50000E94851D10E20E9489090E94661D115073
:103D6000D1F762C161E070E089E00E94851D52C117
:103D700061E070E089E053C169E170E08AE00E948F
:103D8000851D81E08093B805209170058091BD0567
:103D90009091BE05A091BF05B091C005222311F0FE
:103DA000806801C08F778093BD059093BE05A09376
:103DB000BF05B093C00508EB15E0F80181918F01B4
:103DC0000E94661DF5E0013D1F07B9F72DC161E2B4
:103DD00070E08BE00E94851D8091A8048F3F39F030
:103DE0008091A80491E0980F9093A80402C080915C
:103DF000A8040E94661D10E0812F0E94B3150E9446
:103E000009090E94741D1F5F1031B1F70DC161E0F7
:103E100070E08CE00E94851D8091D10503C161E0B6
:103E200070E085E60E94851D89E2E816F10409F03C
:103E3000F8C0D801E4E7F5E08D91819385E0ED3994
:103E4000F807D1F7E7C061E070E086E60E94851DC3
:103E5000EBE1EE16F10409F0E4C0D801EDE9F5E07C
:103E60008D91819385E0E83BF807D1F7D3C061E0FD
:103E700070E087E60E94851D0E943E0DCBC061E088
:103E800070E088E60E94851D85E789838BE1EDE976
:103E9000F5E0DE01129601900D928A95E1F76CE152
:103EA000CE0101960E94DA0B0E94580B83E08093AA
:103EB000710560E273E080E090E00E948F288091BD
:103EC0007105843009F0ADC08FE70E9476090E9429
:103ED00089098983853509F0A4C09CC061E070E040
:103EE0008AE60E94851D89E6898361E0CE010196FC
:103EF0000E94DA0B0E94580B83E08093710560E208
:103F000073E080E090E00E948F28809171058430FA
:103F100009F087C08FE70E9476090E94890989838A
:103F20008E010E5F1F4F7E01EDE1EE0EF11C0E942F
:103F30008909F80181938F01EE15FF05C1F78BE127
:103F4000FE013296ADE9B5E001900D928A95E1F758
:103F50008981893409F065C05DC061E070E08BE65D
:103F60000E94851DF80180818093D2050E94470D33
:103F700051C061E070E08CE60E94851DF0E2EF1612
:103F8000F10461F487E6898380E2F801DE0112968C
:103F900001900D928A95E1F761E203C087E489837D
:103FA00061E0CE0101960E94DA0B0E94580B83E07B
:103FB000809371056CE474E080E090E00E948F28AB
:103FC00080917105843069F58FE70E9476090E941F
:103FD0008909873431F51EC061E070E08DE60E94EA
:103FE000851D89E1E816F104E1F4D801E8EBF5E07C
:103FF0008D91819385E0E13DF807D1F70BC061E039
:1040000070E08EE60E94851DF80180818093D105C5
:104010000E94280D81E006C061E070E08AEC0E94F9
:10402000851D80E00E94661D0E94A21DA196E6E00B
:104030000C94102EA0E0B0E0E0E2F0E20C94F22D3F
:10404000CAECD3E014E606E035E0F32E44E0E42EBB
:1040500053E0D52E62E0C62E80EE95E00E944F2BF5
:10406000892B09F49BC080EE95E00E947C2B282FC1
:10407000809335044091340450E04730510560F797
:10408000FA01EE52FF4F0C941F2E853B29F781E079
:1040900080933404E1CF823609F07DC0C0923404AD
:1040A000DBCF8093330480933204D0923404D4CF96
:1040B0009C013327309331042093300490913204D3
:1040C000982790933204E0923404C6CF382F2227E9
:1040D0004091300450913104242B352B309331041E
:1040E0002093300490913204982790933204F092F8
:1040F00034042536310508F4AFCF61E070E08CEC74
:104100000E94851D81E00E94661D0E94A21D43C081
:1041100020912E0430912F04F901E653FC4F808347
:1041200090913204982790933204C901019690939C
:104130002F0480932E042091300430913104821793
:10414000930708F489CF0093340486CF809132041A
:1041500082130BC060912E0470912F044AEC53E03F
:10416000809133040E94A91D0DC062E070E08BECC9
:104170000E94851D809133040E94661D8091680510
:104180000E94661DFE01812F11928A95E9F7109217
:104190002F0410922E04109234045ECFCDB7DEB7F8
:1041A000E8E00C940E2E81E080936905809169050A
:1041B000882349F080EE95E00E944F2B892BB1F3C4
:1041C0000E941A20F3CF0895AAE2B0E0EAEEF0E2EE
:1041D0000C94F02D0E9460286B017C0181E00E940C
:1041E0007D0A80EE95E00E944F2B892B29F080EE0E
:1041F00095E00E947C2BF5CF2C9811E072E6B72E4B
:10420000E9E2AE2E03E00E9460286C197D098E0958
:104210009F09693C710581059105D0F11123C1F118
:104220000E9460286B017C012B9A80ED97E00E9430
:10423000A807B982E4E7F5E0DE0112968A2D019025
:104240000D928A95E1F76AE2CE0101960E94DA0B9F
:104250002B9880E090E00E94A807009371050E94CF
:10426000580B62E370E080E090E00E948F2880911C
:104270007105843061F4009371058FE70E9476091F
:104280000E94890911E0823419F410E001C011E0A4
:104290008AE00E948529892B81F411E00EC02C9AB6
:1042A0002B9A80EE95E00E947C2B8D309105A9F031
:1042B0005CF40A9791F02C982B9880EE95E00E9480
:1042C0004F2B892B61F79FCF8332910579F0823490
:1042D000910589F70E94D320EECF62EB71E080EE6A
:1042E00095E00E94292A0E943C1DE5CF0E94C71537
:1042F000E2CF8F929F92AF92BF92CF92DF92EF92D6
:10430000FF921F93CF93DF938AE00E948529892B28
:1043100009F089C068EC70E080E090E00E948F288E
:1043200080E090E00E94A8070E9460284B015C0199
:104330006B017C0180ECC80E82E1D81EE11CF11CEF
:104340000E9460286C157D058E059F0530F48AE07B
:104350000E948529892BA1F364C08AE00E948529E7
:10436000892B09F05EC080ED97E00E94A8070E94AB
:1043700060286B017C01D0E0C1E088E4880E86E211
:10438000981EA11CB11C11E08AE00E948529892B8E
:1043900021F58C149D04AE04BF0430F480ED97E049
:1043A0000E94A807D1E0F0CF0E9460286C197D0917
:1043B0008E099F09693C71058105910528F30E94CA
:1043C00060286B017C01C12719F080ED97E002C0E5
:1043D00080E090E00E94A807D7CF80E090E00E94A4
:1043E000A807DD23B9F08091D10590E0019665E042
:1043F00070E00E94932D8093D1050E94280D0E94A9
:10440000A8130E94470D64EF71E080E090E00E94E5
:104410008F2809C080E00E94DF060E94BF110E9421
:104420003E0D0E94E420DF91CF911F91FF90EF900D
:10443000DF90CF90BF90AF909F908F900895CF92D4
:10444000DF92EF92FF9280E00E94DA070E94B107AC
:1044500061E08CE00E94192961E08BE00E9419293B
:1044600060E08AE00E94192960E083E10E94192936
:1044700061E083E10E94522961E082E10E941929F2
:1044800060E082E10E9452290E949F0740E052ECC6
:1044900061E070E080EE95E00E94972C0E94A813E6
:1044A0000E94470D0E9491138FEF8093A8040E94F1
:1044B000C60778940E9460286B017C018091A80453
:1044C0008F3F59F40E9460286C197D098E099F095D
:1044D000603D77408105910588F380ED97E00E946B
:1044E000A80761E08AE00E9452292C9A80EE95E0AC
:1044F0000E944F2B892B29F080EE95E00E947C2BA7
:10450000F5CF6CEF72E080EE95E00E940A2A81E818
:1045100093E00E942F0C63E173E080EE95E00E942F
:104520000A2A4AE050E060E070E080EE95E00E94E8
:10453000DA2A62E370E080E090E00E948F2880EE4B
:1045400095E00E944F2B04970CF180EE95E00E94BD
:104550007C2B82349105D1F480EE95E00E947C2B77
:104560008E34910599F480EE95E00E947C2B843482
:10457000910561F480EE95E00E947C2B819731F4E7
:1045800080E090E00E94A8070E94E4204091750519
:10459000509176056091770570917805DB01CA012D
:1045A0000197A109B1090497A105B10568F44093E9
:1045B000A704433029F440EA56E861E070E004C003
:1045C00040E052EC61E070E080EE95E00E94972CB4
:1045D0000E9479212C9880E090E00E94A8070E9418
:1045E00091131092C3048091BD0583FF11C0809187
:1045F0008905882351F080919005882331F08091BE
:104600009705882311F087E001C085E08093C304FB
:1046100080E00E947D0A8091C4040E94B1090E943A
:10462000580B10923F0410923E0410923D04F12C5E
:104630008091D2058F15B0F062E370E080E090E0E9
:104640000E948F2880ED97E00E94A80762E370E047
:1046500080E090E00E948F2880E090E00E94A80710
:10466000F394E6CF80919C0584FF08C0982F987141
:1046700081E0983109F080E00E947B118FE00E9478
:10468000DA07FF90EF90DF90CF900895EF92FF92BE
:104690000F931F93CF93DF938C016EE770E080EE52
:1046A00095E00E945906E801F12CF0E2EF2E8E0110
:1046B00088818D57823048F46DE770E080EE95E098
:1046C0000E94590688818E2588832196F801608191
:1046D00080EE95E00E94A92BF394F9E0FF12E7CF5A
:1046E0006EE770E080EE95E00E945906CDB7DEB728
:1046F000E6E00C94102EA9E0B0E0E1E8F3E20C94BF
:10470000F82D9091C50491110EC09EEF99838A8374
:104710006B8350E0559547954C832D8319861886F9
:104720001F821E822EC04091CA04842F90E0B4E004
:1047300095958795BA95E1F7242F2F7030E0821771
:10474000930719F18DEF89831B82FE01349650E0A7
:10475000842F90E0A4E095958795AA95E1F7242F02
:104760002F7030E08217930749F0DC01A553BB4F4F
:104770008C918193405F5F5F563051F74093CA043C
:104780005A83CE0101960E9446238091C50490E091
:10479000019666E070E00E94932D8093C5042996EF
:1047A000E2E00C94142EA0E0B0E0E9EDF3E20C940A
:1047B000F12D6C016EE770E080EE95E00E945906E5
:1047C0008601E12CF12CC0E0D0E030E2B32EF801FC
:1047D000608183E8860F823078F46DE770E080EEC8
:1047E00095E00E945906F80160816B2570E080EE2B
:1047F00095E00E94590604C080EE95E00E94A92B26
:10480000E114F10459F0F80180819E01280F311D57
:10481000C901C92FDD27C80FD91FDD273FEFE31AD4
:10482000F30A89E0E816F10459F028E0E216F104F1
:1048300021F48C2F8095F60180870F5F1F4FC7CF23
:10484000CDB7DEB7E9E00C940D2EA9E0B0E0EBE2C5
:10485000F4E20C94F82DE82F362F8091C50490E0F7
:10486000019664E270E00E94932D8093C50458E99C
:10487000598350E15A83813089F048F08230B9F091
:104880008330D9F48B8381EF8C833D8319C085E01D
:104890008B8381EF8C832F5F2D8312C08B8381EFFD
:1048A0008C8384E6489FA00111245D8309C084E0C5
:1048B0008B8381EF8C83ED8303C00E94B81104C009
:1048C000CE0101960E94D3232996E2E00C94142E87
:1048D000A2E0B0E0EEE6F4E20C94ED2D182F762E77
:1048E0002A8349830E946C286B017C018091DB0440
:1048F0008090C6049090C704A090C804B090C904EA
:104900002A8149818823C1F0D701C60188199909F4
:10491000AA09BB094C015D0191EE89169EE2990638
:10492000A104B10420F1241708F4422F202F672D91
:10493000812F0E94252413C0D701C6018819990927
:10494000AA09BB094C015D0191E3891695E7990617
:10495000A104B10460F0672D812F0E947B23C092D7
:10496000C604D092C704E092C804F092C90422960B
:10497000EDE00C94092EA2E2B0E0E1ECF4E20C943C
:10498000EE2D8CE00E94980981110DC06BE173E05F
:1049900080EE95E00E943B2A2C9A80E00E947D0ADE
:1049A0000E94580B2C9880EE95E00E944F2B892B8B
:1049B00001F180EE95E00E947C2B9091A704992351
:1049C00019F00E94BB13EFCF40913E0450E09A01D2
:1049D0002F5F3F4F2F71332760913F0470E0261700
:1049E000370709F3FA01E75BFB4F808320933E040E
:1049F000DACF80917105843009F086C00E946C285E
:104A0000611571058105910549F06093B5047093B6
:104A1000B6048093B7049093B8040CC081E090E092
:104A2000A0E0B0E08093B5049093B604A093B704DF
:104A3000B093B8048091AB049091AC0481609093E2
:104A4000AC048093AB0483E0809371058FE70E94F0
:104A5000760909E614E00E948909F80181938F0123
:104A6000F4E002371F07B9F72091720480916904BE
:104A7000982F922796FF3BC090E492279093720460
:104A8000982F98739833F1F410E0212F30E0809143
:104A90006904877090E0821793074CF11F5F2091A3
:104AA0009C05812F90E0FC01E759FB4F24FF04C0D7
:104AB00080810E949A11E9CF608180EE95E00E948A
:104AC000A92BE3CF8F7399F480916A048093B40487
:104AD00080916B048093B20480916C048093B10444
:104AE00080916F0490E09093AA048093A904809130
:104AF0003D04813019F482E080933D0480913D04AF
:104B0000833011F410923D040E946C286B017C01EB
:104B10008091AD049091AE04A091AF04B091B00427
:104B20000097A105B105C9F0A7019601281B390B13
:104B30004A0B5B0BDA01C901883B9B40A105B1051B
:104B400060F00E94C7098093B3041092AD041092E4
:104B5000AE041092AF041092B0048091B904909109
:104B6000BA04A091BB04B091BC0446015701881A55
:104B7000990AAA0ABB0A84E795E00E94F407861600
:104B80009706A806B90608F4A8C0C092B904D09246
:104B9000BA04E092BB04F092BC040E9457068091D4
:104BA000A8048830A0F08091BD059091BE05A09129
:104BB000BF05B091C0056CE1B695A795979587950F
:104BC0006A95D1F7892B8A2B8B2B09F0A4C1809190
:104BD000A8048F5F8093A8048091B5049091B604D7
:104BE000A091B704B091B8040097A105B105F1F008
:104BF000C81AD90AEA0AFB0A84E795E00E94F4077A
:104C00006C157D058E059F0508F006C18091BD05D8
:104C100084FD04C080ED97E00E94A8071092B504BF
:104C20001092B6041092B7041092B80490917204D6
:104C3000907C9093720450913E0480913F042091A7
:104C40003D04581709F405C1223009F002C19058FB
:104C500090937204E0919C05E770F0E0E758FC4FF8
:104C60006081693008F0DDC0615040E04613DBC070
:104C700080933F0487E3840F90917204892B809383
:104C800072044093400483E080933D042B9A80910A
:104C900081059091C30491112FC10E94780A8091DF
:104CA000C4040E94B109E0919C05E770F0E0E75868
:104CB000FC4F608182E794E00E94930BE091C40472
:104CC000EF5FE093C404E83109F422C1F0E0EC584E
:104CD000FA4F8785882309F41BC10E94020C81309A
:104CE00069F580919C05887149F18091AB049091A0
:104CF000AC04880F991F9093AC048093AB0483E0BD
:104D0000809371050E94580B0E946C286093AD043B
:104D10007093AE048093AF049093B004672B682B1C
:104D2000692B61F481E090E0A0E0B0E08093AD04F5
:104D30009093AE04A093AF04B093B00480919C050F
:104D400084FF1FC08091AB049091AC048E7F0E94C1
:104D50002A09182F6091A9048091B4040E94B1130C
:104D6000482F612F8091B30449A30E94B113009191
:104D7000D205282F49A16091B1048091B2040E940C
:104D800068242B988091C1048130C1F018F08230E2
:104D9000B1F1CEC08AE00E948529892B09F0C8C0F4
:104DA00081E08093C1040E9460286093BD047093E9
:104DB000BE048093BF049093C004BAC08AE00E94EE
:104DC0008529892B31F50E946028C090BD04D090C0
:104DD000BE04E090BF04F090C0046C197D098E09F8
:104DE0009F09693E73408105910508F4A1C082E0E6
:104DF0008093C10480ED97E00E94A80799C08AE0E3
:104E00000E948529892B09F493C080E090E00E94DC
:104E1000A8071092C1048CC080E090E00E94A8070F
:104E200005CF68E022CF851709F422CF4F5F242FEA
:104E300030E090E0F901EE58FB4FDC01A75BBB4F7F
:104E40007C917083F901E05CFB4F708301968F7158
:104E50000DCF2430B1F42091400481E494E0A3E725
:104E6000B4E0FC013E2F381B321718F431913D930A
:104E7000F9CF87E3820F90917204892B809372049B
:104E800002CF8091C104823069F4916090937204E2
:104E90002C9A51ECE52E55E0F52E8E010F5F1F4F39
:104EA000B80110C02C9880913D04811103C081E0AD
:104EB00080933D0480913D04833059F784E08093D2
:104EC0003D04E7CFF70181917F0169A37AA30E9496
:104ED000B315F801819391938F0169A17AA1F1ED46
:104EE000EF16F5E0FF0671F780919C0543E754E06B
:104EF00087700E947908CACE882309F4CECE20910B
:104F0000C20431E0320F3093C2042913C6CE0CC064
:104F10001092C404E2CE8091A804883009F42C9A3F
:104F200089E08093A804D9CE1092C2048150B5CEF6
:104F3000A296ECE00C940A2E8230E8F4E82FF0E020
:104F4000EE0FFF1FED52FA4F71836083813041F005
:104F5000809169008C7F842B80936900E89A089582
:104F600080916900440F551F440F551F837F842B88
:104F700080936900E99A08951F920F920FB60F92DD
:104F800011242F933F934F935F936F937F938F934E
:104F90009F93AF93BF93EF93FF938091D30590912D
:104FA000D405892B29F0E091D305F091D40509951A
:104FB000FF91EF91BF91AF919F918F917F916F91F1
:104FC0005F914F913F912F910F900FBE0F901F90C7
:104FD00018951F920F920FB60F9211242F933F93A3
:104FE0004F935F936F937F938F939F93AF93BF93F1
:104FF000EF93FF938091D5059091D605892B29F0E9
:10500000E091D505F091D6050995FF91EF91BF91FB
:10501000AF919F918F917F916F915F914F913F9150
:105020002F910F900FBE0F901F9018951F920F9207
:105030000FB60F9211242F933F938F939F93AF93AB
:10504000BF938091D8059091D905A091DA05B091D0
:10505000DB053091D70523E0230F2D3720F401968F
:10506000A11DB11D05C026E8230F0296A11DB11D8B
:105070002093D7058093D8059093D905A093DA059E
:10508000B093DB058091DC059091DD05A091DE05F4
:10509000B091DF050196A11DB11D8093DC059093B1
:1050A000DD05A093DE05B093DF05BF91AF919F9121
:1050B0008F913F912F910F900FBE0F901F901895D9
:1050C0002FB7F8946091D8057091D9058091DA05D1
:1050D0009091DB052FBF08953FB7F8948091DC05D0
:1050E0009091DD05A091DE05B091DF0526B5A89B66
:1050F00005C02F3F19F00196A11DB11D3FBF6627C6
:10510000782F892F9A2F620F711D811D911D42E00A
:10511000660F771F881F991F4A95D1F70895CF9280
:10512000DF92EF92FF92CF93DF936B017C010E949D
:105130006C28EB01C114D104E104F10479F00E9460
:105140006C286C1B7D0B683E7340A0F381E0C81A8D
:10515000D108E108F108C851DC4FECCFDF91CF91C5
:10516000FF90EF90DF90CF900895789484B582609F
:1051700084BD84B5816084BD85B5826085BD85B5FB
:10518000816085BDEEE6F0E0808181608083E1E8AA
:10519000F0E01082808182608083808181608083E2
:1051A000E0E8F0E0808181608083E1EBF0E08081E5
:1051B00084608083E0EBF0E0808181608083EAE7B7
:1051C000F0E0808184608083808182608083808140
:1051D000816080838081806880831092C1000895FF
:1051E000833081F028F4813099F08230A1F0089565
:1051F0008630A9F08730B9F08430D1F480918000F6
:105200008F7D03C0809180008F7780938000089508
:1052100084B58F7702C084B58F7D84BD0895809159
:10522000B0008F7703C08091B0008F7D8093B00075
:105230000895CF93DF9390E0FC01ED50F44F24915B
:10524000FC01E95FF34F8491882349F190E0880FD6
:10525000991FFC01E15DF34FA591B4918B5D934FD4
:10526000FC01C591D4919FB7611108C0F8948C914D
:10527000209582238C93888182230AC0623051F466
:10528000F8948C91322F309583238C938881822BD4
:10529000888304C0F8948C91822B8C939FBFDF91FC
:1052A000CF910895A1E0B0E0E8E5F9E20C94F62D85
:1052B000282F30E0F901E152F44F8491F901ED50CB
:1052C000F44F1491F901E95FF34F04910023C9F001
:1052D000882321F069830E94F0286981E02FF0E0A3
:1052E000EE0FFF1FEB5DF34FA591B4919FB7F894BC
:1052F0008C91611103C01095812301C0812B8C9387
:105300009FBF2196E4E00C94122ECF93DF93282FB9
:1053100030E0F901E152F44F8491F901ED50F44F7E
:10532000D491F901E95FF34FC491CC2391F081113D
:105330000E94F028EC2FF0E0EE0FFF1FE55EF34F28
:10534000A591B4912C912D2381E090E021F480E08F
:1053500002C080E090E0DF91CF910895A0E0B0E03E
:10536000E4EBF9E20C94F22D6C017A01EB01E60E0C
:10537000F71E00E010E0CE15DF0561F06991D6015F
:10538000ED91FC910190F081E02DC6010995080F87
:10539000191FF1CFC801CDB7DEB7E8E00C940E2E8F
:1053A0006115710589F0DB010D900020E9F7AD0171
:1053B00041505109461B570BDC01ED91FC910280D5
:1053C000F381E02D0995089580E090E00895EF9233
:1053D000FF920F931F93CF93DF938C01FB01C0E0EB
:1053E000D0E064917F018FEFE81AF80A662361F03C
:1053F000D801ED91FC910190F081E02DC801099553
:10540000C80FD91FF701EDCFCE01CDB7DEB7E6E06B
:105410000C94102E0E94D0290895DC01ED91FC918E
:105420000190F081E02D099508950F931F93CF937C
:10543000DF93EC016DE00E940D2A8C016AE0CE0141
:105440000E940D2A800F911FDF91CF911F910F9124
:1054500008950F931F93CF93DF93EC010E94E729E8
:105460008C01CE010E94152A800F911FDF91CF91F0
:105470001F910F9108950F931F93CF93DF93EC012A
:105480000E94D0298C01CE010E94152A800F911F05
:10549000DF91CF911F910F9108950F931F93CF9399
:1054A000DF93EC010E940D2A8C01CE010E94152A87
:1054B000800F911FDF91CF911F910F910895A1E26D
:1054C000B0E0E5E6FAE20C94EE2D7C01C42EE52F67
:1054D000CB01D22E19A221E02D1510F02AE0D22EF8
:1054E0008E010F5D1F4F8D2C912CA12CB12C6C2D9A
:1054F0007E2FA50194010E94A72D8C2DD29E80198C
:105500001124015011098A3010F4805D01C0895CBA
:10551000F8018083211531054105510521F0C22E86
:10552000E32FCA01E4CFB801C7010E94D029A19698
:10553000ECE00C940A2EA0E0B0E0E1EAFAE20C9470
:10554000F22DEC016A017B012115310541F4E8815E
:10555000F9810190F081E02D642F09951DC02A305A
:105560003105A9F477FF12C06DE20E940D2A8C016B
:1055700044275527BA014C195D096E097F092AE0B5
:10558000CE010E945F2A800F911F06C02AE0B7015A
:10559000A601CE010E945F2ACDB7DEB7E8E00C94E9
:1055A0000E2E9A01AB01662757FD6095762F0E945B
:1055B0009B2A08950F931F93CF93DF93EC019A01D9
:1055C000AB01662757FD6095762F0E949B2A8C01C0
:1055D000CE010E94152A800F911FDF91CF911F915C
:1055E0000F9108952115310549F4DC01ED91FC91ED
:1055F0000190F081E02D642F099508950E945F2AA3
:1056000008959A01462F50E060E070E00E94F22A6F
:1056100008959A01AB0160E070E00E94F22A0895BB
:105620000F931F93CF93DF93EC010E94F22A8C011A
:10563000CE010E94152A800F911FDF91CF911F91FB
:105640000F9108950F931F93CF93DF93EC019A016D
:10565000AB0160E070E00E94F22A8C01CE010E9452
:10566000152A800F911FDF91CF911F910F910895FF
:105670000F931F93CF93DF93EC019A01462F50E0D5
:1056800060E070E00E94F22A8C01CE010E94152A8F
:10569000800F911FDF91CF911F910F910895FC0111
:1056A00024853585F901E05CFF4F80819181F90106
:1056B000EE5BFF4F20813181821B930B8F73992703
:1056C0000895FC0184859585FC01E05CFF4F4081D5
:1056D0005181FC01EE5BFF4F20813181421753075E
:1056E00041F00190F081E02DE80FF91F808190E0FA
:1056F00008958FEF9FEF0895FC0184859585FC0147
:10570000E05CFF4F40815181FC01EE5BFF4F208147
:1057100031814217530779F0A081B181A80FB91FD9
:105720008C91208131812F5F3F4F2F73332731833D
:10573000208390E008958FEF9FEF0895FC0181A1F1
:10574000882329F0A489B5898C9186FFFBCF11A20B
:105750000895CF93DF93FC0126853785D901A05C9E
:10576000BF4F8D919C91119701968F739927E901F5
:10577000CE5BDF4F4881598184179507D9F30D908F
:10578000BC91A02DA20FB31F6C93A685B785A05C1A
:10579000BF4F11969C938E93A689B7892C9181E077
:1057A00090E0078C02C0880F991F0A94E2F7282B1B
:1057B0002C9381E081A30488F589E02D80818064A9
:1057C000808381E090E0DF91CF91089508951F924A
:1057D0000F920FB60F9211242F933F934F938F93F5
:1057E0009F93EF93FF938091C00082FD1CC0409176
:1057F000C600809186069091870601968F7399273F
:1058000020918806309189068217930771F0E09104
:105810008606F0918706EA5BF94F408390938706EE
:105820008093860602C08091C600FF91EF919F9100
:105830008F914F913F912F910F900FBE0F901F901E
:10584000189580EE95E00E944F2B892B11F00E9455
:10585000E62B08951F920F920FB60F9211242F93EB
:105860003F938F939F93EF93FF9320914206309144
:10587000430680914406909145062817390731F474
:105880008091C1008F7D8093C10014C0E0914406D7
:10589000F0914506EE5FF94F20818091440690918A
:1058A000450601968F739927909345068093440689
:1058B0002093C600FF91EF919F918F913F912F917F
:1058C0000F900FBE0F901F901895A0E0B0E0EBE690
:1058D000FCE20C94EE2DFC011382128288EE93E020
:1058E000A0E0B0E084839583A683B7838BEB93E03D
:1058F000918380837587648757874687318B208B98
:10590000138B028BF58AE48AD78AC68AB18EA08E61
:10591000938E828E8F85848F8889858F8989868FE3
:105920008A89878F8B8980A3ECE00C940A2ECF9212
:10593000DF92EF92FF92CF93DF93EC016A017B013C
:10594000411581EE580761057105F9F0EC89FD8973
:1059500081E090E008A002C0880F991F0A94E2F746
:10596000808360E079E08DE390E0A70196010E94DA
:10597000A72D215031094109510956954795379571
:105980002795211580E1380798F0EC89FD89108270
:1059900060E874E88EE190E0A70196010E94A72DCF
:1059A0002150310941095109569547953795279559
:1059B000E889F9893083EA89FB89208319A2EE8975
:1059C000FF89408181E090E09C010C8C02C0220F95
:1059D000331F0A94E2F7422B4083EE89FF8940810E
:1059E0009C010D8C02C0220F331F0A94E2F7422B58
:1059F0004083EE89FF8940819C010E8C02C0220FFA
:105A0000331F0A94E2F7422B4083EE89FF892081FD
:105A10000F8C02C0880F991F0A94E2F780958223A9
:105A20008083DF91CF91FF90EF90DF90CF9008952A
:105A30008F929F92AF92BF92CF92DF92EF92FF929E
:105A40000F931F9381E08F9385E08F9387E08F936F
:105A500083E08F9384E08F93E6EC8E2E912CF2EC12
:105A6000AF2EB12CA1ECCA2ED12CB0ECEB2EF12C28
:105A700004EC10E025EC30E042E056E066E476E02D
:105A800080EE95E00E94652C0F900F900F900F9084
:105A90000F901F910F91FF90EF90DF90CF90BF90EC
:105AA000AF909F908F9008950E94B5280E941F226A
:105AB000C1E2DCE20E94BB242097E1F30E94212C8A
:105AC000F9CFA29FB001B39FC001A39F700D811DAC
:105AD0001124911DB29F700D811D1124911D0895F7
:105AE0000E94612DA59F900DB49F900DA49F800DE5
:105AF000911D11240895B7FF0C94702D0E94702DF4
:105B0000821B930B0895DB018F939F930E94702D4E
:105B1000BF91AF91A29F800D911DA39F900DB29F49
:105B2000900D1124089597FB072E16F4009407D0CA
:105B300077FD09D00E94252E07FC05D03EF49095F4
:105B400081959F4F0895709561957F4F0895A1E2CB
:105B50001A2EAA1BBB1BFD010DC0AA1FBB1FEE1FE7
:105B6000FF1FA217B307E407F50720F0A21BB30B32
:105B7000E40BF50B661F771F881F991F1A9469F7AE
:105B800060957095809590959B01AC01BD01CF010A
:105B90000895052E97FB1EF400940E94E02D57FDFA
:105BA00007D00E94A72D07FC03D04EF40C94E02DE3
:105BB00050954095309521953F4F4F4F5F4F089539
:105BC00090958095709561957F4F8F4F9F4F089569
:105BD0002F923F924F925F926F927F928F929F92FD
:105BE000AF92BF92CF92DF92EF92FF920F931F93EB
:105BF000CF93DF93CDB7DEB7CA1BDB0B0FB6F8949C
:105C0000DEBF0FBECDBF09942A88398848885F84DB
:105C10006E847D848C849B84AA84B984C884DF804C
:105C2000EE80FD800C811B81AA81B981CE0FD11D30
:105C30000FB6F894DEBF0FBECDBFED010895EE0F95
:105C4000FF1F0590F491E02D0994AA1BBB1B51E1A5
:105C500007C0AA1FBB1FA617B70710F0A61BB70BDC
:105C6000881F991F5A95A9F780959095BC01CD0181
:105C700008958F929F92AF92BF92CF92DF92EF9250
:105C8000FF92CF93DF93EC01688179818A819B81B8
:105C9000611571058105910521F464E279ED8BE5CB
:105CA00097E02DE133EF41E050E00E94C92D49011A
:105CB0005A019B01AC01A7EAB1E40E94702D6B016F
:105CC0007C01ACEEB4EFA50194010E947E2DC60EBE
:105CD000D71EE81EF91EF7FE06C081E0C81AD108DB
:105CE000E10880E8F80AC882D982EA82FB82C7010B
:105CF000B6019F77DF91CF91FF90EF90DF90CF902B
:105D0000BF90AF909F908F9008950E94392E089574
:105D100086E091E00E94392E089560930601709309
:105D20000701809308019093090108952F923F92F3
:105D30005F926F927F928F929F92AF92BF92CF921B
:105D4000DF92EF92FF920F931F93CF93DF938B011C
:105D5000EA016115710521F0DB018C9311969C938A
:105D6000209739F09E01225031092332310508F085
:105D7000D8C07C016701BFEFCB1ADB0A5601F701DF
:105D80006080862D90E00E94C82F892B11F076014B
:105D9000F1CFFDE26F120AC0570182E0A80EB11CDC
:105DA000D70111966C90772473940BC0BBE26B12F1
:105DB00007C05701E2E0AE0EB11CD70111966C90FE
:105DC000712CCE018F7E892B89F4B0E36B1237C022
:105DD000F50180818F7D8835D1F46180F2E0AF0ECE
:105DE000B11C872D8260782EC0E1D0E0CA30D10589
:105DF00051F1C031D10521F0C830D10599F409C065
:105E0000CC24CA94DC2CEC2CAFE0FA2E22C02097D4
:105E100069F7C8E0D0E0CC24CA94DC2CEC2CFFE17C
:105E2000FF2E17C06FEF7FEFCB019E01442737FD98
:105E30004095542F0E94A72D69017A010AC020972E
:105E4000A9F6CAE0D0E0E9E9CE2EDC2CEC2CE9E1A1
:105E5000FE2EF50160E020E030E0A9014E01AA2409
:105E600097FCA094BA2C1F0170ED572E560CA9E098
:105E7000A51570F48FEB860D8A3118F499EC592E24
:105E800006C08FE9860D8A3148F589EA582E560CEE
:105E9000852D90E08C179D070CF56F3FD9F0C21649
:105EA000D306E406F50698F0C501B4010E94832DDF
:105EB0009B01AC01852D90E0A0E0B0E0280F391FD8
:105EC0004A1F5B1F281739074A075B0710F46FEF5B
:105ED00001C061E03196D1016C90C5CF011511056B
:105EE00051F0662311F0319703C071FE04C0329760
:105EF000D801ED93FC9370FE07C050954095309506
:105F000021953F4F4F4F5F4F67FF10C082E290E0F7
:105F100090938B0680938A066FEF7FEF8FEF9FEF52
:105F200007C060E070E080E090E002C0B901CA0103
:105F3000DF91CF911F910F91FF90EF90DF90CF9065
:105F4000BF90AF909F908F907F906F905F903F90A9
:105F50002F900895FC0188279927E89421912032F9
:105F6000E9F3293010F02E30C8F32B3241F02D32F6
:105F700039F4689404C00E94FC2F820F911D219176
:105F800020532A30C0F31EF4909581959F4F0895B9
:105F9000911150C0803219F089508550D0F7089582
:105FA00048EC53E00E94D52F0895FA01A191B081E9
:105FB000009719F41097E1F0CD01DC01CD010D90AF
:105FC000002011F4C00113C0FB012191222319F01C
:105FD0002015D9F7F3CFFB012191201519F41E925A
:105FE000119606C02223C1F70D900020A1F7D00121
:105FF000FA01A193B08308957AE0979F902D879F2F
:10600000802D910D11240895F999FECF92BD81BD87
:10601000F89A992780B50895262FF999FECF1FBACF
:1060200092BD81BD20BD0FB6F894FA9AF99A0FBEC1
:0E60300001960895992788270895F894FFCFC8
:10603E0000008C06200001000000FF00020002009C
:10604E000200020002000200020002000200020032
:10605E00020002000200020002000280250000057C
:10606E00400AA1204EA50020244EA52C2330C0129C
:10607E0000001A400AA1204EA5001B1E27522C23F9
:10608E00308025000005400AA1204EA50020244E98
:10609E00A52C2330004B000006400AD0009D49007D
:1060AE007B289D492C233000E1000005400A450164
:1060BE00D7DC03B81E0EBF00232E48E801008A402D
:1060CE000A6001555502AD1E20000023C854582009
:1060DE0074696D656F75742100596573004E6F009C
:1060EE002C00386368004E2F41002C205B005D2091
:1060FE0028002900486F70206368616E6E656C2001
:10610E000020402000456E746572696E67206164E0
:10611E00617074697665206368616E6E656C20735C
:10612E00656C656374696F6E2C207069636B696E44
:10613E00673A007363616E6E6572206D6F64650001
:10614E004E4F5420454E41424C45440053656E64BB
:10615E00696E672073657474696E677320746F203F
:10616E0052580A00526573657474696E67207365C0
:10617E007474696E6773206F6E2052580A00416204
:10618E006F727465642065646974730A00696E7653
:10619E00616C69642073656C656374696F6E000D64
:1061AE000A496E76616C696420696E707574202D73
:1061BE0020646973636172646564210700536574BA
:1061CE0074696E677320736176656420746F204501
:1061DE004550524F4D0A00526576657274656420C3
:1061EE0073657474696E67732066726F6D204545B2
:1061FE0050524F4D0A004C6F6164656420666163B6
:10620E00746F72792064656661756C74730A004BE5
:10621E00657920616E64206368616E6E656C7320B3
:10622E0072616E646F6D697A65640A004F70656E97
:10623E004C52536E67205458207374617274696E99
:10624E00672000206F6E20485720006D6F64756CBC
:10625E0065206C6F636B65643F00342B340038002F
:10626E00382B340031320031322B340031360050AD
:10627E00504D0052535349005344410053434C0078
:10628E00525844005458440041494E004C42454532
:10629E00500053504B54524D0053425553005355DA
:1062AE004D44004C4C494E440000070B0C10111588
:1062BE0000B6012A032E033003340337033C03B622
:1062CE00013F03430348034C035003540358035C3C
:1062DE0003620369036E0373038C028C028C028CBF
:1062EE0002160A1322312900000000A92BAE294FF5
:0862FE002B7C2B612B9E2B0071
:107E00000F92CDB7DEB7112484B714BE81FFF1D035
:107E100082E08093C00088E18093C10086E0809377
:107E2000C20080E18093C4008EE0CDD088249924E4
:107E3000CC24C394F5E0DF2EE1E1EE2E73E0F72EC3
:107E4000B6D0082F813479F4B2D08983C2D0898129
:107E5000823811F481E005C0813811F485E001C059
:107E600083E09ED09AC0823411F484E103C085344B
:107E700019F485E0B6D091C0853561F498D0082F0B
:107E800010E095D090E0982E8824802A912A880CC2
:107E9000991C82C0863521F484E0A3D080E0E1CF34
:107EA000843609F04CC083D082D0A82E80D0B82E62
:107EB00000E011E07CD0F80181938F01AE16D1F77C
:107EC00088D0FB2DF53489F4E0E0F1E00BC0F9999E
:107ED000FECF92BC81BC0894811C911C819180BD15
:107EE000FA9AF99AEA1598F358C08B2D863409F05E
:107EF00054C0F401F7BEE89507B600FCFDCFF401CD
:107F0000A0E0B1E02C9130E011968C91119790E0B7
:107F1000982F8827822B932B12960C01C7BEE895C9
:107F20001124329681E0A038B80761F7F401D7BE7A
:107F3000E89507B600FCFDCFE7BEE8952EC0843774
:107F4000F1F435D034D0182F32D0B82E42D0FB2DDA
:107F5000F63421F4F40105914F010CC0FB2DF534EA
:107F600049F4F999FECF92BC81BC0894811C911C04
:107F7000F89A00B5802F14D0115049F70EC08537FC
:107F800039F427D08EE10CD085E90AD08FE069CF93
:107F9000813511F488E017D01CD080E101D050CF9A
:107FA0009091C00095FFFCCF8093C600089580910A
:107FB000C00087FFFCCF8091C00084FD01C0A89560
:107FC0008091C6000895E0E6F0E098E19083808318
:107FD0000895EDDF803219F088E0F5DFFFCF84E10E
:107FE000DFCF1F93182FE3DF1150E9F7F2DF1F9166
:0E7FF0000895282E80E0E7DFEE27FF27099492
:027FFE0001057B
:0400000300007E007B
:00000001FF
